:1000000085C09FC06BC29DC09CC09BC09AC099C058
:1000100098C034C896C095C094C093C092C091C097
:1000200090C08FC08EC028C72EC73EC710C70FC74D
:1000300050C70DC70CC70BC70AC709C708C707C7F2
:1000400006C705C757C75CC75FC764C76AC772C71B
:1000500078C704C778C702C776C775C774C704C70F
:10006000F6C6F5C6F4C6F3C6F2C6F1C6F0C6EFC6CC
:10007000EEC6EDC6ECC6EBC6EAC6E9C6E8C680C762
:1000800004030904120345006E00740072006F003F
:1000900044006500760016035500530042002D0011
:1000A000410056005200490073007000084156524A
:1000B0004953505F32001201010102000008C016CE
:1000C000E105000101020001090243000201008074
:1000D00019090400000102020100052400100104B6
:1000E00024020205240600010524010301070583FB
:1000F0000308006409040100020A0000000705016A
:1001000002080000070581020800000011241FBE3C
:10011000CFE5D4E0DEBFCDBF10E0A0E6B0E0E0E781
:10012000F2E102C005900D92AE38B107D9F713E0A5
:10013000AEE8B0E001C01D92AE31B107E1F709D8D9
:1001400096C85ECF85B78C6085BF8BB780688BBF44
:1001500083EC8093EE028093E30208951F93DC0109
:10016000162F8091630084FF11C08091E30298E80C
:1001700089278093E302912F91509F3F59F0E4EE3D
:10018000F2E08D9181939150E0F704C08AE580936D
:100190006300F1CF612F84EE92E09CD11C5F10933D
:1001A00063001F9108951F93DC01162F8091620058
:1001B00084FF11C08091EE0298E889278093EE02B7
:1001C000912F91509F3F59F0EFEEF2E08D91819386
:1001D0009150E0F704C08AE580936200F1CF612F6F
:1001E0008FEE92E077D11C5F109362001F9108950B
:1001F0000F931F93CF93DF936091FE02161634F591
:1002000063508091FB02CEE0D3E0C81BD1098091FE
:10021000FA028F3F09F48DC08D3209F450C08091ED
:100220008E0087FD0BC0CE01F5D78F3F09F484C047
:10023000882309F072C02FEF30E002C020E030E8E0
:1002400030938E00209360001092FE028091610036
:1002500084FF29C0809160008F3F29F1682F893089
:1002600008F051C0861B8093600080918E0080FF53
:1002700052C003EC8F5F80938E0087FD65C06623BC
:1002800009F44EC089ED92E0D8D7682F7727162F52
:10029000693008F475C08FEF809360009EE1009391
:1002A000D802909361009AE080B38C7009F0F4C09A
:1002B0009150D1F71092FF021092F902EDC08AE539
:1002C00080936100683009F0B9CF8881807609F0A9
:1002D0006EC021EE32E01092E1028981882309F09C
:1002E00075C01092E2023093FD022093FC0222E0DE
:1002F00030E88F81882309F0A3CF8E81821708F020
:100300009FCF282F9DCF68E0861B8093600080914F
:100310008E0080FDAECF0BE4ADCF20E030E090CF7B
:1003200060E089ED92E0D6D094E08FEF809360009A
:10033000B6CFCE0162D788CF809360008EE18093E4
:1003400061002FEF30E07CCF2091FC023091FD0264
:1003500086FD1FC0462F41504F3F61F0F901942F99
:10036000A9EDB2E081918D939150E0F7240F311DFA
:100370002F5F3F4F3093FD022093FC02772787CFFA
:1003800089ED92E0A7D0912F9C5F183008F087CFBD
:10039000CCCF462F41504F3F69F3F901942FA9ED7F
:1003A000B2E084918D9331969150D8F7DFCFCE0192
:1003B000BBD6282F30E82F3F09F09BCF888187FDDF
:1003C00002C03F773DCF2E813F773ACF853069F02D
:1003D000863089F08830D9F0893011F18A3071F196
:1003E0008B3021F120E030E884CF8A818093FF02B6
:1003F00020E030E87ECF8B81813039F1823029F1E5
:10040000833041F1813209F120E030EC72CF81E09C
:1004100093E09093FD028093FC0221E030E869CFE5
:100420008A818093010320E030E863CF83EC8093DE
:10043000EE028093E30220E030E85BCF3093FD02D0
:100440002093FC0221E030E854CFCE0152D6282F71
:1004500030ECB1CF8A81882349F480E890E0909312
:10046000FD028093FC0224E030EC43CF813059F050
:10047000823051F686E990E09093FD028093FC0271
:1004800026E130EC36CF84E890E09093FD02809333
:10049000FC0222E130EC2DCFDF91CF911F910F9123
:1004A0000895A82FB92F8FEF9FEF41E050EA6150D8
:1004B00070F02D9138E0722F7827969587952695C4
:1004C00070FF02C0842795273A95A9F7F0CF809551
:1004D00090950895E6DF8D939D930895CF93CFB7C0
:1004E000CF93829BFECF829B09C0829B07C0829BD9
:1004F00005C0829B03C0829B01C09EC0DF93C09158
:10050000FB02DD27CE5FDC4F829B02C0DF91EBCF89
:100510002F930F931F9300B32FEF02FB20F94F93FC
:100520003F9310B34FEF012702FB21F93BE031C0AD
:100530004E7F012F10B3216028C0102F4D7F226005
:10054000000000B329C04B7F2460012F000010B3CE
:100550002BC010B3477F28602AC04F7E00B32061B4
:100560002CC04F7D10B320622FC04F7B00B320649E
:1005700032C0422700B349934FEF0000102712FB0F
:1005800020F910B31C70A9F1297F91F2012702FB19
:1005900021F900B3237F89F23150F0F1102712FBCB
:1005A00022F910B3277E79F2012702FB23F92F7C71
:1005B00081F200B3102712FB24F92F7971F200C0E9
:1005C00010B3012702FB25F92F7359F200C000B3C5
:1005D000102712FB26F9223040F200C010B3012789
:1005E00002FB27F9243028F64F77206810B300006B
:1005F000F9CF3B503195333010E81ABFB8F0C31B28
:10060000D0400881033C99F10B3489F11981412FC5
:100610001F772091F902121731F40936E9F10D32F2
:10062000C1F0013EB1F02227209300033F914F918A
:100630001F910F912F91DF91CF91CFBFCF9118953F
:100640003091630034FD56C000936300C3EED2E0E6
:1006500055C047FD0FEF009300033F914F911F914D
:100660000F912F91DF91CAB7C7FD3BCFE5CF009126
:1006700000030023D9F21091FE021123B9F53430A2
:10068000BAF13093FE020093FA021091FB023BE0B4
:10069000311B3093FB022CC00091FE02013034F577
:1006A0000AE547FD09C03091610034FD23C0009385
:1006B0006100C8EDD2E022C01A8110FDC1CF309197
:1006C000620034FD17C000936200CEEED2E016C087
:1006D000052710E002BB1FC0052722C0052727C041
:1006E00005272CC0052710E002BB33C04AE503C034
:1006F00042ED01C0432FC4E1D0E032E011B31C60F1
:10070000929A02B311BB5F935CE020E820FF0527BB
:1007100002BB279517951C3FD8F620FF0527279584
:1007200002BB17951C3FC0F620FF0527279517959C
:1007300002BB1C3F98F620FF0527279517951C3F05
:1007400002BB70F600C0499120FF052702BB279528
:1007500017951C3F38F620FF0527279502BB1795F4
:100760001C3F38F520FF05272795179502BB1C3F36
:1007700010F520FF0527279517951C3F02BBE8F4CD
:10078000242F3A9519F6037F5F9102BB00C01091A8
:10079000FF02C651D04011F01093F90210E81ABFC1
:1007A000046011B3137F402F437F02BB11BB42BBD8
:1007B0003DCF0527D3CF0527D8CF0527DDCFFC01B7
:1007C00050918F00F89435B33F7E919148E097FDAA
:1007D0001EC035BB789422B72195251B82B7820FA6
:1007E00087FDFCCFF894AA9A990F3F7E9B99916060
:1007F000789422B72195251B82B7820F87FDFCCF05
:10080000F894AA98415019F76150F9F602C0306186
:10081000E0CF7894892F90E0089564E0D0DF80E005
:1008200090E00895FF920F931F93CF93DF938C0175
:10083000EC012196FC016081CE01C1DFF82EF801A8
:100840000081043030F464E0601BCE01800F911D04
:10085000B6DF8F2D90E0DF91CF911F910F91FF9028
:1008600008958F929F92AF92BF92DF92EF92FF9284
:100870000F931F93CF93DF93EC014B018881FA8094
:100880008F1508F4F82E93E0A92EB12CAC0EBD1EE6
:100890006F2DC50194DF84010F5F1F4FEF2CFF24E4
:1008A000888190E08E199F09181619068CF5AE0CF8
:1008B000BF1CDD2420E030E061E0C9018A0D9B1DF2
:1008C0007EDF982F8981D81618F4F80191938F0153
:1008D000A895D3942D2D30E0888190E08E199F0942
:1008E000281739074CF38981D816A0F480E9E82E3F
:1008F00080E0F82E1092900061E0C70160DFF801FF
:1009000081938F01A895D3948981D81698F302C05A
:10091000DD24E9CFF4011082F8011082898190E092
:100920000296DF91CF911F910F91FF90EF90DF9092
:10093000BF90AF909F908F9008958F929F92AF92AB
:10094000BF92CF92DF92EF92FF920F931F93CF93BC
:10095000DF93EC014B01E42E10929300442321F429
:1009600080911B0387FD39C0D880C98084010F5F47
:100970001F4FF4011082FA80C114D104E1F1C0E0EC
:10098000D0E020E9A22E20E0B22E10C0C0FD1BC096
:1009900087EFF822F092900064E0C50110DFF801C3
:1009A00081938F012196CC15DD0589F0A895809162
:1009B0001903809391008091180380939200EE2098
:1009C00029F3C6D1E7CFF8E0FF2AC2D1E3CF8601F1
:1009D000080D191D0F5F1F4F0EC08DE4809390000E
:1009E0001092910080911A038093920064E080E954
:1009F00090E0E5DEB9CFF8011082C6010296DF91E2
:100A0000CF911F910F91FF90EF90DF90CF90BF900B
:100A1000AF909F908F900895A298A498A398AA98B9
:100A2000AC98AB98AD985FD385B58F7E85BDAD9AF8
:100A3000C598C49A08950F931F938C01FC0180817F
:100A4000EBDFF80181814FD31F910F910895CF9370
:100A5000DF9341D3C0E9D0E080EF80939000109203
:100A6000910064E0CE01ABDE80FF07C080911C03E3
:100A7000882391F781E890E002C080E090E0DF9168
:100A8000CF9108954F925F926F927F928F929F9233
:100A9000AF92BF92CF92DF92EF92FF920F931F938C
:100AA000CF93DF93EC01062F988019818A8180FF14
:100AB00071C070E2572E60E4462E002321F480912D
:100AC0001B0387FD71C0812E7E01CC24DD2430E91B
:100AD000A32E30E0B32E34010894610871080BC0D6
:100AE000C614D70410F097FD6FC00894C11CD11C28
:100AF0000894E11CF11CC814D90409F452C0A8954B
:100B00008091190380939100809118038093920043
:100B1000F7018185809393001C81002351F5177F95
:100B2000C0FC35C01093900064E0C50148DE9A8196
:100B300090FDD6CF892F8521F1F0F70111858F81A6
:100B4000811711F188858117F9F08E81877FC0FCAC
:100B500026C0809390008B81BED264E0C5012FDE59
:100B6000811719F280911C038823B9F780E890E07F
:100B700033C0EED0D7CF942139F08B8168DF882342
:100B800009F4B3CF90E028C08B81ADD2AECF18600E
:100B9000DFD0C8CF54E0552E48E0442E8ECF886079
:100BA000D8CF80E090E018C08DE480939000109240
:100BB000910080911A03809392001092930064E058
:100BC00080E990E0FCDD7FCF8D818093900064E030
:100BD000C501F5DD9A81AECFDF91CF911F910F91C5
:100BE000FF90EF90DF90CF90BF90AF909F908F904D
:100BF0007F906F905F904F900895FF920F931F9397
:100C00008C01FC01F08064E00296D9DDF80181815D
:100C1000882351F0F9E0FF1520F48F2D18DF90E0C4
:100C200007C0EAE0FE2EF9CF8F2D5DD280E090E084
:100C30001F910F91FF900895DF92EF92FF920F9313
:100C40001F93CF93DF93EC01298190917C00C59A8B
:100C5000C498992309F057C0B19960C0B19B5AC09C
:100C6000892F82958F7096959695980F9F5F909398
:100C70008F0085B38B7E85BB84B3846184BBAD98C4
:100C800085B5806185BD822F2ED220918F0092B7CD
:100C90009195921B82B7890F87FDFCCFAD9A92B7D1
:100CA0009195921B82B7890F87FDFCCFAD988A8101
:100CB0001AD2D0908F000FE1F7E0EF2EF12CEC0E5E
:100CC000FD1EA8956E81C7017ADD182F8E818430B4
:100CD00058F18D81181791F1AA9A92B791959D19A3
:100CE00082B7890F87FDFCCFAA9892B791959D197D
:100CF00082B7890F87FDFCCF015018F780E08CDEAA
:100D000080EC90E01DC0913061F0923051F0933052
:100D100009F0A4CF83E080938F00ABCF10928F00B7
:100D2000A8CFB19B9BCFA3CF64E0681B9701280F8E
:100D3000311DC90144DD8D81181771F680E090E006
:100D4000DF91CF911F910F91FF90EF90DF90089569
:100D50008091180390911903A0911A03B0911B037D
:100D60000196A11DB11D8093180390931903A093C0
:100D70001A03B0931B0308959C018BE18093B1018A
:100D8000809195008093B2013093B3012093B40118
:100D90008EE08093B5011092CB021092CA02C90175
:100DA00006969093CD028093CC02019759F0E1EB27
:100DB000F1E090E02A543E4F81919827E217F30723
:100DC000D9F703C0E1EBF1E090E0908308958091C2
:100DD000CC029091CD022091CA023091CB02821BAD
:100DE000930B08952091CC023091CD02211531054D
:100DF000D9F08091CA029091CB02FC01EF54FE4FD2
:100E0000E08101969093CB028093CA0282179307E8
:100E100040F01092CD021092CC021092CB021092B0
:100E2000CA028E2F90E008958FEF9FEF0895CF9321
:100E3000DF93C2E0D0E0809199008093B6011092D8
:100E4000B70190E0FC013197ED32F10520F080EC24
:100E50008093B70195C0ED5EFF4F09948AE990E059
:100E6000DCDC8093B7018CC067EB71E08AE990E02D
:100E7000F8DCEC01219684C06CEA70E088EB91E02C
:100E8000EFD1CBE07DC020919B00E0919A00E63944
:100E900009F466C0E73909F46AC0F0E0EF71F07058
:100EA000EC59FF4F20836CC0E0919A00EA3909F4B5
:100EB00053C0E63909F45DC0E73909F45FC0F0E0DA
:100EC000EF71F070EC59FF4F80818093B801C3E05F
:100ED00057C080919A0080931B0380919B00809360
:100EE0001A0380919C008093190380919D00809348
:100EF000180346C08AE990E09FDE8093B70140C0A6
:100F00008AE990E098DD3CC08AE990E076DE809343
:100F1000B70136C060E08AE990E0B4DD8093B701A4
:100F20002FC040E067EB71E08AE990E006DDEC015C
:100F3000219626C061E08AE990E0A4DD8093B701A4
:100F40001FC041E0EFCF8AE990E06CDC8093B801EC
:100F50001092B901C4E014C089EC8093B70110C0AD
:100F600085B5922F9770887F982B95BD96CF23BD1E
:100F700094CF85B590E087709070A7CF83B5A5CF4B
:100F8000CE01FADEDF91CF910895482F80911D03A5
:100F9000882341F41092AE011092AD014B3109F05B
:100FA00069C042C08091AD019091AE010097B1F34C
:100FB00021E08931920708F042C0DC01AC56BF4FF6
:100FC0004C939C012F5F3F4F3093AE012093AD01B6
:100FD00024303105C9F12530310579F1253031054D
:100FE00008F448C08091AF019091B00128173907EB
:100FF00009F040C090E0E4E9F0E09D012F5F3F4F31
:1010000081919827E217F307D9F71092AE01109259
:10101000AD01992371F180EB8093B6018093B70104
:1010200082E090E0A9DE26C04093940081E090E049
:101030009093AE018093AD011DC04E30D9F0109257
:10104000AE011092AD0116C0809197008093AF0160
:10105000809196008093B0018091AF019091B00192
:1010600006969093B0018093AF018A51914038F772
:1010700001C0DDDE88EC80931D03089578941F92F3
:101080000F920FB60F9211248F93F89480911C0346
:10109000882329F080911C03815080931C0378944D
:1010A000F89480918400815080938400882361F4B7
:1010B00089E48093840080911D03882329F0809126
:1010C0001D03815080931D0378948F910F900FBE64
:1010D0000F901F901895982F96959695891B8F5F66
:1010E00080931C030895F7DF80911C038823E1F7A8
:1010F0000895FC018091D702882341F483818130D7
:1011000051F028EC30E083E490E009C020E030E0CA
:1011100080E090E004C026EB30E082E190E0309384
:10112000FD022093FC020895FC01808180768032CC
:1011300019F080E090E008958091D7028823C9F7E4
:10114000818180528230A8F71092D6028FEF90E012
:101150000895EF92FF920F931F93CF93DF9388E14F
:1011600090E02EE00FB6F894A89581BD0FBE21BD8A
:1011700082E188BB80E387BB88E085BB84E384BBD6
:1011800012BA8CE081BB11BA83E083BF81E089BFD2
:1011900089E085BD82E083BDD5D778940091D702E0
:1011A0008EECE82E82E0F82EA89522D80023E1F7F5
:1011B0008091620084FFF8CFC0E0D0E01C2F12DEE7
:1011C00097FD0FC0FE01E253FD4F8083612F6F5FDB
:1011D0002196C830D10591F760938500C701E3D708
:1011E000E3CF6C2FCC23C1F7809185008823E1F2F7
:1011F00060938500C701D7D7D7CF1F93CF93DF93D5
:10120000EC01162F8991C1DE1150E1F7DF91CF91EA
:101210001F9108959C018091D602882359F48BE494
:101220008093EE02A6E8B0E0F90187E001900D920C
:101230008150E1F781E090E008959C018091D60211
:10124000882359F4F901A6E8B0E087E00D900192F7
:101250008150E1F787E090E0089580E090E0089504
:10126000FB01DC0105900D920020E1F70895FFCF0E
:10127000FF5A5A5A00000000000000000000000061
:101280000000000001020A0032000180000000009E
:0E1290000000000001018025000000000800A1
:00000001FF
